:100000002500A3048F0C0200020C0600010C260040
:100010006700040026070F0A07061F0A090A0604DC
:100020000706190A07050602040F26002909060516
:10003000090A86053309E70586040605090A410908
:10004000090AFF0C2800040000000000E802230A4F
:10005000000804001E0C2900FF0C2A00EA022E0AE8
:10006000E9022C0A0008FF0C2900FF0C2A000400FA
:100070000000000000000000EA02370AE902350A29
:100080000008E707480AFF0C2900FF0C2A00E704D4
:10009000EA020008E9024E0A67000008FF0C2A0085
:0200A000000856
:021FFE000E00D3
:00000001FF
